:020000040000FA
:100000008316860181168312930164309400930B4A
:100010000728940B0728810105180C28930B0C283E
:100020008A01010844208E000108532090008C00B2
:10003000010862208F000108712091008D0080303E
:10004000930010088C0B25288C0011088D0B292893
:100050008D0002308A000C080E020022920003304C
:100060008A000D080F02002312078600000000001E
:10007000000000000C0B3D28930B21288601051C75
:100080003F28930B3F2804288207F934F934483479
:1000900048344834893489348934C434C434C43449
:1000A000F934F934F9348207353435344834483476
:1000B00048344134413441343B343B343B343534AF
:1000C0003534353482077034703429344E3470340A
:1000D00029344E34703429344E3470344E3429343B
:1000E00070348207223422342934253422342934CE
:1000F0002534223429342534223425342934223439
:100400008207403445344B34503455345B346034C7
:10041000643469346D347134743477347A347C34B0
:100420007D347E347F347F347F347E347D347B343E
:1004300079347734743470346C34683464345F34B1
:100440005A3455344F344A3444343F3439343434D4
:100450002E34293424341F341A34163412340E3412
:100460000B340834053403340234003400340034CF
:100470000034013402340434063409340C340F34AB
:10048000133417341C34213426342B3430343634AE
:100490003B34403446344C34523458345D34633445
:1004A00068346C347034743477347A347C347E3409
:1004B0007F347F347F347E347D347B3479347634BA
:1004C00072346E346A34653460345A3455344F347F
:1004D000493442343C34363430342A3424341F34E2
:1004E0001A34153411340D3409340634043402340A
:1004F000003400340034003401340334053408344B
:100500000B340F34133418341D34223428342E3471
:1005100034343A34403446344D3454345A346034EC
:1005200066346B347034743478347B347D347E3488
:100530007F347F347F347D347B3479347534713447
:100540006D34683462345C3456344F344934423448
:100550003B3434342E34273421341B3416341134D4
:100560000C340934053403340134003400340034CD
:1005700001340334053408340C34113416341B347C
:10058000213427342D3434343B34403447344E3412
:1005900056345D34633469346F34733477347B3468
:1005A0007D347F347F347F347E347C3479347634C8
:1005B00071346C34673460345A3453344B344434BB
:1005C0003C3435342D3426342034193413340E346D
:1005D0000A34063403340134003400340034023465
:1005E000043407340B34103415341B3421342834CC
:0405F0003034373438
:10060000820740344A3453345C3465346C34733478
:1006100078347C347F34803480347E347B34763458
:1006200071346A3462345934503447343D3433348D
:100630002A342134193412340C340734033401348D
:1006400000340134033406340B34113419342134AA
:100650002A3433343D3440344B3455345F346834B9
:10066000703476347B347E34803480347E347A3413
:1006700074346E3465345C34523448343D3432342E
:1006800028341E3416340E34083404340134003453
:100690000134033408340D3415341D342734313417
:1006A0003B3440344C34573462346B3473347934D3
:1006B0007E34803480347D34793473346B346134E7
:1006C00056344B343F34333428341D3414340C3412
:1006D0000634023400340034033407340E34163444
:1006E00020342A34363440344D345A3465346F342F
:1006F00077347C347F3480347E3479347234683497
:100700005D345134443437342A341E3414340B34B9
:10071000053401340034013406340C3415341F34EC
:040720002B3438340A
:02400E00FA3F77
:00000001FF
